:10607200011900001D01010C0200000301FA0400D5
:10608200FA0500030A0A5A0B001E0C00FA0D00035F
:106092000E00040F0164100096120132130AFA1462
:1060A200010215010217010A1801FA1905321A0133
:1060B2000A1B01FA1C05321FFFFF20FFFF23011EEE
:1060C2002400642A00FA2B00FA2C50782D003C2E72
:1060D20000462F001E300064325078330000343204
:1060E200FA350164360164370150380A643C0064B1
:1060F2003E003C3F000140FFFF411450420A5A4318
:106102000AC84405324500B44600FA47011848025D
:10611200034C00FA4EFFFF500404510596520A3216
:10612200530B46540A965601025705465800025927
:106132000A465A32FA5B010A5C0A325E000A5F00C2
:10614200FE61FFFF64010666000267FFFF6A0A3C08
:106152006B00006C32967300007400007801327993
:1061620001327EFFFF81FFFF84FFFF8500AF8600C3
:10617200018700FA89010A8A00009900009D0A96A7
:106182009E00019FFFFFA0FFFFFAFAFA00001D0127
:10619200010C0200000301FA0400FA0500030A0AD6
:1061A2005A0B001E0C00FA0D00030E00040F0164CE
:1061B200100096120132130AFA1401021501021795
:1061C200010A1801FA1905321A010A1B01FA1C0503
:1061D200321FFFFF20FFFF23011E2400642A00FA62
:1061E2002B00FA2C50782D003C2E00462F001E303A
:1061F20000643250783300003432FA3501643601DB
:1062020064370150380A643C00643E003C3F0001A0
:1062120040FFFF411450420A5A430AC8440532451E
:1062220000B44600FA47010C4802024C00FA4EFF45
:10623200FF500404510596520A32530B46540A96F3
:10624200560101570546580001590A465A32FA5B6F
:10625200010A5C0A325E000A5F00FE61FFFF640110
:106262000666000267FFFF6A0A3C6B00006C32960A
:106272007300007400007801327901327EFFFF81E1
:10628200FFFF84FFFF85FFFF86FFFF87FFFF890176
:10629200028A00009900009D0A969E00019FFFFF5E
:1062A200A0FFFFFAFAFA0065006F00790083008D03
:1062B200009700A100AC00B600C000CA00D400DE06
:1062C20000E800F20058006000680070007800806A
:1062D20000880090009800A000A800B000B800C19B
:1062E20000C800D000D800DF00E600EE00F6004152
:1062F2000047004D00530059005F0065006C0071BB
:106302000077007D00830089008F0095009B00A22A
:1063120000A700AC00B200B900C000C500CA00D29C
:0A63220000D500DD00E100E700EF08
:103A3900900043E0D3940440149007B4E0FEA3E05F
:103A4900FF906074126465E493F59980129007B44D
:103A5900E0FEA3E0FF90618E126465E493F599900E
:103A690007B4E0FEA3E0FF906072E493FC74019355
:103A7900FDEFB50507EEB50403754D009007B412C7
:103A8900644C2285F97385FA747E017F00E574120E
:103A9900643EE5732FFF50010E8E5A8F5B90001321
:103AA900E0FCA3E0FDEF2DFDEE3CFC8C5C8D5D227E
:103AB90075A71085F97385FA747E017F00E5741284
:103AC900643EE5732FFF50010E8E5A8F5B9000D62E
:103AD900E0B40210AC2CAD2DEF2DFDEE3CFC8C5C5E
:103AE9008D5D8016AE5AAF5B900013E0FCA3E0FD3C
:103AF900EF2DFDEE3CFC8C5C8D5D22AE5AAF5B7404
:103B09001E8E048F05FF12642E8C5C8D5DAE5AAF3C
:103B19005B741E8E048F05FF1264598C5A8D5BE508
:103B29005B455A6013741EC3955BFFE4955AFE8E7C
:103B39005A8F5B785C126492E573A85CB80015D360
:103B4900955D4010E573C3955DFFE4955CFE8E5C61
:103B59008F5D8010E573240CC3955DFFE4955CFED1
:103B69008E5C8F5D22900084E0B40104C212800251
:103B7900D212900085E0B40104C2138002D21390DE
:103B890000C2E075F0D2A4FFAEF0740A8E048F056E
:103B9900FF12642E9007AAECF0A3EDF0A20D4016D7
:103BA90074038C068D0712643E7401120039900764
:103BB900A8EEF0A3EFF07E017F00900080E0126490
:103BC9003E9000C3E08E048F05FF12642E740AFF35
:103BD90012642E8D609000CCE075F0D2A4FFAEF097
:103BE900740A8E048F05FF12642E9007AEECF0A3C1
:103BF900EDF09000CEE060139000CEE0F5F0741681
:103C090084FF7E00EF9007BCF0800674649007BCC7
:103C1900F09000C4E0900068F090010EE09000522E
:103C2900F090009DE0900054F09000C6E09000559F
:103C3900F0900072E0900056F09000F8E090005B80
:103C4900F090015CE090005CF090015DE090005D17
:103C5900F090015EE090005EF0A229B34016900159
:103C69005CE0700C90015DE0700690015EE060021E
:103C79008002C22974E3900067F09000ADE0B40BB4
:103C89000874E3900067F0805A9000ADE0B419120F
:103C99009000C3E090629312008CE493900067F067
:103CA90080419000ADE0B41E129000C3E09062B173
:103CB90012008CE493900067F080289000ADE0B486
:103CC90028129000C3E09062DB12008CE49390000C
:103CD90067F0800F9000ADE0B446089000A4E09032
:103CE9000067F09000DDE0FE9000ABE06E600A90A6
:103CF90000ABE09000DDF0D22890006BE0FE900070
:103D0900AAE0B5063390006DE0FE9000C8E0B50664
:103D19002790006CE0FE9000D6E0B5061B90006F7E
:103D2900E0FE90007DE0B5060F90006EE0FE900089
:103D3900B8E06E7003023E81900043E0C3940550E1
:103D49000874029000F9F080149000D6E0600874BD
:103D5900089000F9F08006740A9000F9F090007D4F
:103D6900E0B4010674009000E3F090007DE0B40235
:103D79000674009000C8F090007DE0B4030674005A
:103D89009000D5F09000C8E0D394014014741890C5
:103D990000FBF074009006C2F074009006C3F08036
:103DA9000C74009000FBF074189006C2F09000AA01
:103DB900E06014741A900091F074009006CAF074CF
:103DC900009006CBF0800C7400900091F0741A906A
:103DD90006CAF09000AAE0B402147419900092F097
:103DE90074009006C6F074009006C7F0800C740049
:103DF900900092F074199006C6F09000D6E0700E0B
:103E090074059006D6F074069006DAF080187400EE
:103E19009006D6F074009006D7F074009006DAF098
:103E290074009006DBF0D2289000AAE090006BF0B5
:103E39009000D6E090006CF09000C8E090006DF022
:103E49009000B8E090006EF090007DE090006FF077
:103E590090007DE0900053F09000B8E0900057F09A
:103E69009000D6E0900058F09000AAE0900059F038
:103E79009000C8E090005AF09000E0E0B40117907B
:103E8900001F740FF0A374FFF0900021E4F0A3F079
:103E990074029000E0F09000E0E0B403419000214A
:103EA900E0FEA3E0FF90001FE0FCA3E0FD12648A9E
:103EB900741012643E7408120039EF900064F0EF38
:103EC900700674FF900064F074009000E0F09000B8
:103ED90020E0900065F090001FE0900066F09000EF
:103EE90071E0900037F0900037E02406900038F038
:103EF900900038E0D3940C400B900038E0C3940C48
:103F0900900038F0900071E0FE9000D4E02E90000F
:103F19003CF090003CE0D3940C400B90003CE0C393
:103F2900940C90003CF090003CE0D39406400D9036
:103F3900003CE0C3940690003DF0800A90003CE00C
:103F4900240690003DF09000B7E0900039F0900011
:103F590039E0D3940C400F900039E0C3940C9000E1
:103F690039F0D2228002C222900039E02406900062
:103F79003AF090003AE0D3940C400B90003AE0C339
:103F8900940C90003AF022C293C294C291C292C298
:103F990087C290E5B554EFF5B5E5B554DFF5B5C27F
:103FA90096C295C2A0C297C2A2C2A1E5B554BFF5F7
:103FB900B5E5B5547FF5B5E5B554FBF5B5C214754E
:103FC9005E469000BAE07005756D028003756D0359
:103FD90075550075540090000874FFF0A374DCF067
:103FE900C219C21B74C8900033F074C8900035F030
:103FF900755300755200C20D754600E56FB409038B
:10400900756F00756300900015E4F0A3F0757010EA
:10401900C217C2189007AAE0FEA3E0FF7403126456
:104029003E74011200399007A8EEF0A3EFF0C20226
:1040390075570075560090000CE4F0A3F0C22A757C
:10404900590075580090007CE075F032A4FDACF081
:1040590090001DECF0A3EDF0C23AA22EB39205A296
:104069002FB39206A230B39207A231B39208A232BB
:10407900B39209A233B3920AA234B3920BA235B315
:10408900920C2285F97385FA747E017F00E574121A
:10409900643EE5732FFF50010E8E5A8F5BAC5CAD09
:1040A9005DEF2DFDEE3CFC8C5C8D5DD293D294E5E9
:1040B9005DF5FBE55CF5FCE55DF5E9E55CF5EA90A8
:1040C90000B8E0B40314D291D292E55DF5EBE55C5A
:1040D900F5ECE55DF5EDE55CF5EE2275A71085F9E2
:1040E9007385FA747E017F00E57412643EE5732FCF
:1040F900FF50010E8E5A8F5B7E017F769000F5E0AE
:1041090012643EAC5AAD5BED2FFFEC3EFE8E5C8F28
:104119005DE55DF5FDE55CF5FE900068E4F075A7E9
:1041290000741290003FF02285F97385FA747E01BC
:104139007F00E57412643EE5732FFF50010E8E5A1D
:104149008F5B9007AAE0FCA3E0FDEF2DFDEE3CFCA0
:104159008C5C8D5DE55DF5FDE55CF5FE220564226F
:104169009000B8E0B403539000D6E0B4012EA2D871
:10417900B34004C293C287A2D9B34004C294C29087
:10418900A2DAB34008C291E5B554EFF5B5A2DBB3A5
:104199004008C292E5B554DFF5B5801CA2D8B340FA
:1041A90002C293A2D9B34002C294A2DAB34002C2B6
:1041B90091A2DBB34002C292801EA2D8B3400AC2C8
:1041C900939000D6E06002C287A2D9B3400AC29494
:1041D9009000D6E06002C290A2DCB34004C296C24D
:1041E9009575D8402285A77275A710A2D8B3400249
:1041F900C287A2D9B34002C290A2DAB34006E5B59C
:1042090054EFF5B5A2DBB34006E5B554DFF5B5A229
:10421900DCB340089000C4E0900068F075D8408590
:1042290072A722900047E4936406600280FE74C876
:104239009007B0F8E4F0E8A3F075B500758401754E
:10424900A70075FFA090003BE4F075C91075A70F92
:1042590075A1C775A70075D90075CE0C75A70F751F
:10426900F1FE75F2FF75F30775F47875A4BA75A5B3
:10427900FF75A60775AE0075AFFF75D48175D5FFBB
:1042890075D6FF75D7FF75A70075A20175A147758A
:10429900F80975D80075D90475DA0975DB0975DC73
:1042A9000975DD0975DE0975D84075A71075D8003F
:1042B90075D90475DA0975DB0975DC0975DD0975C8
:1042C900DE0975D84075A70075E60875E71075BC55
:1042D9000175BE0475BD6C75BE0775BDA075BE08B8
:1042E90075BD0175BC0075BB1875BC2075BA08751C
:1042F900E88075D11375A70F75E10575E20075C7DB
:1043090040123F90759700759780740A12641E7564
:1043190097C0E5975420700280F8758F0275A70041
:10432900D2AF75980075A90C75A70F75AB4375AD1C
:10433900FB75AC1E75A71075C91875CA0075CB0039
:1043490075C80475A700758912758E04758C00757A
:104359008A00C2A9D28C758D00758B00D2ABD28E22
:1043690075EF0675D944C29974C8F5097508001224
:1043790000E975B5001204E974639007B0F8E4F038
:10438900E8A3F012037574C89007B0F8E4F0E8A345
:10439900F07464F5097508001200E9900053E09083
:1043A900007DF090007DE0D39403400C74009000F0
:1043B9007DF07400900053F0C21F90007DE0905C86
:1043C90086F82828738028A2B44002D21F8020755D
:1043D900A70F75F30F75A700A2A34002D21F800F84
:0F43E90075A70F75F31775A700A2A44002D21F86
:0C5C86000243CE0243D00243D80243E99F
:1043F800A21FB3405F757308E573D3940E5020E590
:10440800739007B0F8E4F0E8A3F01202447464F57E
:10441800097508001200E97873740126F650D974FA
:10442800029000B9F0900053E090007DF090007D7C
:10443800E0905C92F8282873801674009000E3F0EE
:10444800800E74009000C8F0800674009000D5F0CB
:0C5C920002444002444202444A024452D0
:10445800D21E805D757301E573D394075020E57310
:104468009007B0F8E4F0E8A3F01202447464F50988
:104478007508001200E97873740126F650D97401A2
:104488009000B9F0900053E090007DF090007DE03E
:10449800905C9EF8282873801674009000E3F080E2
:0F44A8000E74009000C8F0800674009000D5F0EC
:0C5C9E0002449F0244A10244A90244B148
:1044B700C21E900052E090010EF0900053E0900071
:1044C7007DF0900054E090009DF0900055E0900042
:1044D700C6F0900056E0900072F0900057E0900010
:1044E700B8F0900058E09000D6F0900059E09000A6
:1044F700AAF090005AE09000C8F090005BE09000AE
:10450700F8F090005CE090015CF090005DE09001B5
:104517005DF090005EE090015EF090015CE0700C51
:1045270090015DE0700690015EE060028004C229A0
:104537008002D2299000C3E07006740A9000C3F08D
:104547009000A4E0700674E39000A4F09000AAE045
:104557000490006BF09000ABE09000DDF0123B6E32
:10456700E5B54401F5B57406900041F0740190007B
:1045770042F07403900044F07405900045F07423F2
:10458700900046F07405900047F0900043E0B404B3
:10459700067404900047F07401900048F07400908E
:1045A700004DF07400900050F074FF900051F074CB
:1045B70032900147F07434900148F0742B90014910
:1045C700F0745490014AF0744490014BF074439096
:1045D700014CF0742090014DF0743490014EF0744A
:1045E7004390014FF07479900150F0746C90015131
:1045F700F07420900152F07420900153F0742090D1
:104607000154F07420900155F09000DFE0900064B1
:10461700F0900096E0900065F0900097E0900066BB
:10462700F0A2B6B39210A2B3B39211C20EC20FA2F8
:10463700A4B39225A2B4B39226A2A3B39227900063
:1046470060E4F0756F00743A900770F074FD90079E
:1046570071F0900061E4F09007AAE0FEA3E0FF7418
:104667000312643E74011200399007A8EEF0A3EF1D
:10467700F0756E0190003FE4F0C224756300C21527
:10468700D216C202757100C22CD203C22DD204C247
:104697002ED205C22FD206C230D207C231D208C2EB
:1046A70032D209C233D20AC234D20BC235D20CC2BB
:1046B70020C221C222C223C22812009E755F007544
:1046C7006B00756100756532756600756700756802
:1046D70000756900756A00900015E4F0A3F0756C29
:1046E70000D2B2D2A4D2B0D2B1D2A3D2A7D2A6D28C
:1046F700A5D2B790007CE0D394FA400674FA9000F4
:104707007CF07E017F00900066E012643E900065B9
:10471700E02FFF50010E90001FEEF0A3EFF0EFD354
:1047270094FFEE940F400790001FE4F0A3F0900071
:1047370064E0700674FF900064F09000B9E0D394D1
:1047470002400674019000B9F09000BAE070057558
:104757006D028003756D039000BBE0D394014006A2
:1047670074009000BBF09000C1E0C3940A50067437
:104777000A9000C1F09000CBE0700674019000CB66
:10478700F09000CBE0B4FF0674FE9000CBF09000F1
:10479700D2E0D394FE400674FE9000D2F09000F869
:1047A700E0D39402400674019000F8F090010EE007
:1047B700D394014006740190010EF074019000D863
:1047C700F074019000D9F074009000E0F07400904C
:1047D70000FCF07400900100F074299006B6F074A4
:1047E7002A9006BAF074179006BEF0741B9006CE96
:1047F700F0741C9006D2F0D29C9000ABE0D39404E6
:10480700400674049000ABF0E570D3941040037534
:1048170070109006B7E0D3940C400674009006B76A
:10482700F09006BBE0D3940C400674009006BBF0F2
:104837009006BFE0D3940C400674009006BFF0903A
:1048470006C3E0D3940C400674009006C3F09006AC
:10485700C7E0D3940C400674009006C7F09006CBCF
:10486700E0D3940C400674009006CBF09006CFE09E
:10487700D3940C400674009006CFF09006D3E0D393
:10488700940C400674009006D3F09006D7E0D394BA
:104897000C400674009006D7F09006DBE0D3940C2A
:1048A700400674009006DBF0D2EC75CF01A298B3F6
:1048B7004005C298120646E54D6006A299B3B3407B
:1048C700028005C299120C57E54E64016005E54E5A
:1048D700B4040280D5C28E7E107F00E56412643E68
:1048E700E58D75F010A4FDACF0EF2DFDEE3CFCE579
:1048F7008B75F01084FF7E00ED2FFFEC3EFE8E548B
:104907008F55D28E90009DE0605C90001712644C2A
:10491700900017E0FCA3E0FD900019E0FAA3E0FB8C
:10492700EDB50342ECB5023EB21DA20DB3401975B9
:10493700E700A21DB34008E5B54404F5B58006E5D8
:10494700B554FBF5B575E710900019E0FEA3E0FF3D
:1049570090001BE0FCA3E0FDEF2DFDEE3CFC90007A
:1049670019ECF0A3EDF09000AAE060099000AAE02E
:10497700C394034002806F122D96A20DB350099085
:104987000060E0C3941C40028006900094E0F54567
:10499700E54575F005A4FFAEF09007B2EEF0A3EF82
:1049A700F0900081E0C395614007E55FC3956050D3
:1049B700079007B2E4F0A3F0AE2EAF2F9007B2E056
:1049C700FCA3E0FDEFD39DEE9C4004C2A1800B90B9
:1049D7000060E0C3942A5002D2A19000AAE0B4027A
:1049E70005A2A1B392A29000AAE0B4031C122EB1B3
:1049F700AE2EAF2F9007B2E0FCA3E0FDEFD39DEE04
:104A07009C4004D2A18002C2A1900085E06009A267
:104A1700B3301101B3B340028059A2B3301101B3CF
:104A27004051A2B3301301B3403C9000B8E0B40347
:104A370006A220B3B340028006740490003FF0D270
:104A470020A214B3401BD20EC20FE55E640C6005B2
:104A5700E55EB41802800AE56D7006740390003FA6
:104A6700F0A213B39211A213B330B301B34004A25F
:104A7700139211A2B6301001B350030250C0A2B670
:104A8700301001B350030250C0A2B6301201B35028
:104A970003024F04756E00055EA20EB35003024B6E
:104AA700F3E56DB40354A22AB34048E55E640D6094
:104AB70005E55EB41903756D01A20F401CE55EC3E1
:104AC700940D500690003F7401F0E55ED3940D40BD
:104AD70006740290003FF0801AE55EC394195006F1
:104AE70090003F7401F0E55ED3941940067402907C
:104AF700003FF0755E01D22A805CE56DB402067551
:104B07006D01755E0DE55EB40D05755E018047901C
:104B1700003FE07032E55EC3940D500690003F748D
:104B270001F0E55ED3940D4006740290003FF0E576
:104B37005EC3940D5002D224E55ED3940D4002D299
:104B470024C296C295C2A09000BAE0B40105123FF4
:104B5700908003755E01C20E90009DE06043900057
:104B670017E0FEA3E0FF90009DE08E048F05FF1283
:104B7700642E74018C068D0712003990001BEEF02D
:104B8700A3EFF090001BE0F8A3E0900019C8F0A392
:104B9700C8F0900017E4F0A3F0C21DE5B554FBF58B
:104BA700B5A2B4B34002C226A2A4B34002C225A252
:104BB700A3B34002C227A224B34002C224A220B357
:104BC7004006A22292218002B221900085E0601265
:104BD700E56D700EA220B35009A221302201B3B3B4
:104BE70040028006740590003FF0C220A20FB35028
:104BF70006E55E640D60028050755E01D20FA2B4B7
:104C0700B34002C226A2A4B34002C225A2A3B34066
:104C170002C227A224B34002C224A220B34006A2A4
:104C27002292218002B221900085E06012E56D702A
:104C37000EA220B35009A221302201B3B340028053
:104C470006740590003FF0C220A20FB3B35006E5EB
:104C57005E640D60028012740590003FF0D22490CC
:104C670000BAE0B40103123F90AE58AF59AC54AD4F
:104C770055EF2DFDEE3CFC8C588D59AE54AF55EFDA
:104C8700D39DEE9C401190000FE0FAA3E0FBEBC32D
:104C970094E8EA94034002800690000F12644C9057
:104CA700000CE0FEA3E0FFAC54AD55EF2DFDEE3C4C
:104CB700FC90000CECF0A3EDF0AE56AF57AA54AB46
:104CC70055EF2BFBEE3AFA74018A068B071200396F
:104CD7008E568F57AC54AD55EDD39498EC943A401B
:104CE70003123F90C28E758D00758B007564007539
:104CF7005501755400D28EE55E75F00384AFF07EE2
:104D070000EF4E707590000CE0F8A3E090000AC821
:104D1700F0A3C8F090000AE0FEA3E0FFEF4E600B9F
:104D27007C7B7D2212632C8E528F5390000CE4F013
:104D3700A3F0AE52AF537428BE00039F5010E56333
:104D47002FFF50010E74011200398E528F53855375
:104D5700639000C1E0A852B8000DD395534008E511
:104D67005390003EF080099000C1E01490003EF09F
:104D7700E56D60067553007552009000B8E0B40306
:104D870008900039E0655E6002800BA221B3400401
:104D9700D2238002B223E55E64066005E55EB40CAB
:104DA700099000AAE060031223D290003CE0655E00
:104DB700600790003DE0B55E03756F00A215B35024
:104DC70006A214B3B34003024E76900076E0B40116
:104DD700739000F8E0B40214120E26900069E07593
:104DE700F0BEA4FFAEF08E5C8F5D8056E56775F070
:104DF7000A84FF7E00900570126465E0F55B755AC2
:104E070000AE5AAF5B90009BE012643E74648E0460
:104E17008F05FF12642E8C5C8D5DE55D90000EF0B2
:104E2700AE5AAF5B900074E012643E74648E048FD8
:104E370005FF12642E74BE8C068D0712643E8E5CCD
:104E47008F5D8017900074E075F0BEA4FFAEF08E02
:104E57005C8F5D90009BE090000EF0E561C394CC01
:104E67005006E55D455C7002800312408CD215E563
:104E77006DB40106E55E64046002800975700190F7
:104E870000407401F0E56D706F9000BDE0600D901B
:104E97000068E0A852B80006955340028038900099
:104EA700BDE0B40217900037E0655E6007900038F8
:104EB700E0B55E03757003756C00800CC200756CFD
:104EC70000900015E4F0A3F0900068E06006740914
:104ED70090003FF08022900037E0B55E0B757001BF
:104EE7009000407401F08010900038E0B55E0975BD
:104EF70070017402900040F0A212B39210A212B394
:104F070030B601B350030250C0756E01E5B54401D8
:104F1700F5B5741C900060F0A2129210E55ED39470
:104F27004A4014D214E55ED39460400B7405900098
:104F37003FF0D224755E469000C5E0B40107E56AEC
:104F4700C3941440028009123F90741390003FF0FD
:104F5700A22C300301B3501D75E700A22CB3400803
:104F6700E5B54408F5B58006E5B554F7F5B575E739
:104F770010A22C9203A22D300401B3501D75E70037
:104F8700A22DB34008E5B54402F5B58006E5B55452
:104F9700FDF5B575E710A22D9204A22E300501B3D9
:104FA700500FA22EB34004D2A08002C2A0A22E921C
:104FB70005A22F300601B3500FA22FB34004D2979A
:104FC7008002C297A22F9206A230300701B3500F7A
:104FD700A230B34004D2A28002C2A2A2309207A29A
:104FE70031300801B3500FA231B34004D2A180027F
:104FF700C2A1A2319208A232300901B3501D75E750
:1050070000A232B34008E5B54440F5B58006E5B5E2
:1050170054BFF5B575E710A2329209A233300A01E1
:10502700B3501D75E700A233B34008E5B54480F5DA
:10503700B58006E5B5547FF5B575E710A233920A3A
:10504700A234300B01B3500FA234B34004D287808F
:1050570002C287A234920BA235300C01B3500FA2C3
:1050670035B34004D2908002C290A235920CE56A13
:10507700C394415009740E90003FF0123F90900086
:1050870047E0FE900043E004C39E4009900043E0E0
:10509700D39408400974FB90003FF0123F909000B2
:1050A7004CE0601590004CE0FE900046E06E600911
:1050B70074FE90003FF0123F90A224B34004C296C2
:1050C700C2959000F5E0600CAE52AF537414BE0069
:1050D700059F4002804890007DE0905CAAF8282850
:1050E70073803BA2B4B35005A226B34002800512D9
:1050F70040E4D2268028A2A3B35005A227B34002DA
:1051070080051240E4D2278015A2A4B35005A2253A
:0E511700B3400280051240E4D22580028000E1
:105CAA000250E80250EA0250FD025110025123024A
:025CBA00512572
:10512500A217B3B35008900039E0655E60030252E0
:1051350004A201B35006A200B3B34003025200908B
:1051450000B8E0B4030280030251D5A20DB3406755
:10515500A223B3402D123A8CE55DF5FBE55CF5FC29
:10516500D293A202B34002D2879000D6E0B40210D7
:10517500123AB9E55DF5FBE55CF5FC75A700D2874C
:105185008033123A8CE55DF5EBE55CF5ECD291A246
:1051950002B34006E5B54410F5B59000D6E0B4027B
:1051A50014123AB9E55DF5EBE55CF5EC75A700E59C
:1051B500B54410F5B58017123A8CE55DF5FBE55C55
:1051C500F5FCE55DF5EBE55CF5ECD293D291802B32
:1051D500123A8CE55DF5FBE55CF5FCD293A202B3D2
:1051E5004002D2879000D6E0B40210123AB9E55DCC
:1051F500F5FBE55CF5FC75A700D287C217D218A2AE
:1052050018B3B3500890003AE0655E60030252E3BC
:10521500A201B35006A200B3B340030252DF9000CF
:10522500B8E0B4030280030252B4A20DB34067A2F2
:1052350023B3402D123A8CE55DF5E9E55CF5EAD23C
:1052450094A202B34002D2909000D6E0B4021012AC
:105255003AB9E55DF5E9E55CF5EA75A700D2908018
:1052650033123A8CE55DF5EDE55CF5EED292A202DE
:10527500B34006E5B54420F5B59000D6E0B4021478
:10528500123AB9E55DF5EDE55CF5EE75A700E5B516
:105295004420F5B58017123A8CE55DF5E9E55CF536
:1052A500EAE55DF5EDE55CF5EED294D292802B1240
:1052B5003A8CE55DF5E9E55CF5EAD294A202B340E6
:1052C50002D2909000D6E0B40210123AB9E55DF52D
:1052D500E9E55CF5EA75A700D290D217C218E5702A
:0E52E500905CBCF82828730256B79000ABE02E
:065CBC000252EC0252EF5F
:1052F300905CEFF8282873121EAE8012121EAE8047
:0E5303000D121F388008121FE48003121FE4F1
:0F5CEF000252FA0252FF02530402530902530EEB
:105311007570020256B7122110122227A23AB34029
:105321002290009FE0F56C900070E0256CFE9000EB
:105331003EE075F01E84FC7F00EE2CF53674109073
:10534100003FF09007A8E0FEA3E0FF740A12643E5C
:1053510090000AE0FCA3E0FD74098F02FF12642EA5
:105361008D078C038E048A058B0612632C9007AC83
:10537100EEF0A3EFF09000C6E0B401087478BE002F
:10538100059F4002800D74789007ACF8E4F0E8A323
:10539100F0801B9007ACE0FEA3E0FF74F0BE0003B9
:1053A1009F500B74F09007ACF8E4F0E8A3F0E536F9
:1053B10070037536019007ACE0FEA3E0FFE5362FE0
:1053C100FF50010E9007ACEEF0A3EFF07570039063
:0353D1000040E0B9
:035CC20002531773
:1053D400905CFEF82828738010A23B400375700A85
:0953E4008007A23B400375700B29
:095CFE000253DB0253DD0253E600
:1053ED000256B79006B7E060031224EA9000F6E08B
:1053FD00B401149000F7E0A852B80004955350077B
:10540D00E55FC3956040028009741590003FF0027E
:10541D0054A09000ABE0D39402403F90007FE02475
:10542D0003A852B8000495535009900081E0D3951C
:10543D006150028008D201740890003FF090007F07
:10544D00E0A852B80005D39553500B900081E0248D
:10545D0003C395615002C201803990007FE024039F
:10546D00A852B8000495535007E55FC395604002FC
:10547D008008D201740890003FF090007FE0A852A0
:10548D00B80005D395535009E560240FC3955F50BF
:10549D0002C2019000C5E07007E56AC39414400292
:1054AD008002D201A2014005757004800A7570104A
:1054BD00900015E4F0A3F0A20DB34029E56775F057
:1054CD000A84FF7E00900570126465E0C3946950F4
:1054DD0005122407800F9007AAE0F8A3E09007A813
:0C54ED00C8F0A3C8F00256B79000ABE076
:065CC5000253F00254F549
:1054F900905D07F8282873120F108012120F108080
:0E5509000D1210BE8008121170800312117076
:0F5D070002550002550502550A02550F025514A8
:105517009006BBE060031225C67570050256B712E8
:1055270012B07570069006BFE060031226B69006AB
:10553700C3E060031227920256B790000EE06006A0
:10554700A20DB3B34002801D90000EE02529FFAEE7
:105557002850010E8E288F29E55ED39406500690B9
:10556700000EE014F01214F67570079006C7E0609D
:105577000312286E9006CBE0600312294A0256B741
:105587009000F8E0B40203120E9E1218F575700829
:105597009006CFE06003122A269006D3E06003123C
:1055A7002B020256B7121CB1A217B35005A218B3AB
:1055B70040028004D217D2187570109006D7E060A9
:1055C70003122BDE9006DBE06003122CBA0256B7FB
:1055D7000256B7900034E0C394465008C29674460A
:1055E700900034F085365B755A00900037E0F5730C
:1055F700123B04E55D900034F0900004E55AF0A3F7
:10560700E55BF0C21A9007ACE0F55AA3E0F55B90B2
:105617000037E0F573123B04E55D900033F090002E
:1056270000E55AF0A3E55BF0C219E56DB401057515
:10563700700B80037570038077900036E0C3944643
:1056470050139000C6E0B40104C2968002C295745C
:1056570046900036F085365B755A00900038E0F5C5
:1056670073123B04E55D900036F0900006E55AF0B2
:10567700A3E55BF0C21C9007ACE0F55AA3E0F55B2D
:10568700900038E0F573123B04E55D900035F0902B
:105697000002E55AF0A3E55BF0C21BE56DB4010318
:1056A700756D007570038008800680048002800095
:105CCB000255260255410255870255AC0255D702A3
:105CDB0055DA0256400256AF0256B10256B302567F
:045CEB00B50256B7F1
:1056B700900033E0B55E60A219403C900000E0FE28
:1056C700A3E0FFEF4E602EAC56AD577405FF126492
:1056D7002E8D068C07900000E0FCA3E0FDCFCECF17
:1056E70012000374068E048F05FF12642E900000CB
:1056F700ECF0A3EDF0D219AE54AF55900000E0FCEA
:10570700A3E0FDEFC39DEE9C400D124131D296C23E
:105717001974C8900033F0A219B3B350079000333F
:10572700E0B55E02800D124131D29674C890003305
:10573700F0C219900034E0B55E5DA21A403C9000BB
:1057470004E0FEA3E0FFEF4E602EAC56AD577405A4
:10575700FF12642E8D068C07900004E0FCA3E0FD89
:10576700CFCECF12000374068E048F05FF12642E6E
:10577700900004ECF0A3EDF0D21AAE54AF559000B0
:1057870004E0FCA3E0FDEFC39DEE9C400AC29674C3
:1057970046900034F0C21AA21AB3B35007900034EF
:1057A700E0B55E02800AC2967446900034F0C21AD1
:1057B700900035E0B55E6BA21B403C900002E0FE16
:1057C700A3E0FFEF4E602EAC56AD577405FF126491
:1057D7002E8D068C07900002E0FCA3E0FDCFCECF14
:1057E70012000374068E048F05FF12642E900002C8
:1057F700ECF0A3EDF0D21BAE54AF55900002E0FCE5
:10580700A3E0FDEFC39DEE9C40181241319000C606
:10581700E0B40104D2968002D295C21B74C89000EE
:1058270035F0A21BB3B35007900035E0B55E028098
:10583700181241319000C6E0B40104D2968002D21A
:105847009574C8900035F0C21B900036E0B55E68CD
:10585700A21C403C900006E0FEA3E0FFEF4E602E46
:10586700AC56AD577405FF12642E8D068C07900059
:1058770006E0FCA3E0FDCFCECF12000374068E0432
:105887008F05FF12642E900006ECF0A3EDF0D21CFA
:10589700AE54AF55900006E0FCA3E0FDEFC39DEECC
:1058A7009C40159000C6E0B40104C2968002C295E0
:1058B7007446900036F0C21CA21CB3B35007900088
:1058C70036E0B55E0280159000C6E0B40104C296CA
:1058D7008002C2957446900036F0C21C9000C8E062
:1058E700B4020280030259FF900062E0D39566502C
:1058F70064900062E0F4042566FE9000CBE08E0021
:10590700F5F0E884FF7E008F73EFC39410500CEF1F
:105917008573F0A4FDACF08D7380037573FF900061
:1059270062E0D39573400B900062E0C39573F57105
:1059370080037571009000E6E0D3957140069000F2
:10594700E6E0F5719000E7E0C3957150069000E737
:10595700E0F5718071900062E0C39566FE9000CB20
:10596700E08E00F5F0E884FF7E008F73EFC394109C
:10597700500CEF8573F0A4FDACF08D738003757345
:10598700FF85735B755A00900062E0255BFFAE5A96
:1059970050010E8E5A8F5B74FFBE0009D39F4005DE
:1059A700855B7180037571FF9000E6E0D3957140C8
:1059B700069000E6E0F5719000E7E0C395715006A8
:1059C7009000E7E0F571A20DB3B3500D900063E0CE
:1059D700FE9000D3E0D39E5002800A740790003FE8
:1059E700F0C297801375A710E5CDC395714004C227
:1059F700978002D29775A700E56FC39409500AA252
:105A0700EDB34005C2ED123050AE54AF557498C394
:105A17009F743A9E400C900061E0C3945A40030281
:105A27005C83A214B34009123F90740690003FF0C4
:105A3700A21FB34008E5B54404F5B58006E5B554A3
:105A4700FBF5B5A216B3500EE561D394334007E5D5
:105A570061C394CC400280419000F8E0B402141274
:105A67000E26900069E075F050A4FFAEF08E5C8FB3
:105A77005D800F900074E075F050A4FFAEF08E5C6F
:105A87008F5DE55D455C6011E5B54401F5B5741CB6
:105A9700900060F012408CD216900061E0D3940120
:105AA7004007E561C3941A40028002C2169006B708
:105AB700E060031224EAA22C300301B35017A22C92
:105AC700B34008E5B54408F5B58006E5B554F7F5E4
:105AD700B5A22C92039006BBE060031225C6A22D47
:105AE700300401B35017A22DB34008E5B54402F5C1
:105AF700B58006E5B554FDF5B5A22D92049006BF15
:105B0700E060031226B6A22E300501B3500FA22E75
:105B1700B34004D2A08002C2A0A22E92059006C371
:105B2700E06003122792A22F300601B3500FA22F75
:105B3700B34004D2978002C297A22F92069006C75D
:105B4700E0600312286EA230300701B3500FA23075
:105B5700B34004D2A28002C2A2A23092079006CB21
:105B6700E0600312294AA231300801B3500FA23175
:105B7700B34004D2A18002C2A1A23192089006CFFD
:105B8700E06003122A26A232300901B35017A2326D
:105B9700B34008E5B54440F5B58006E5B554BFF513
:105BA700B5A23292099006D3E06003122B02A2330A
:105BB700300A01B35017A233B34008E5B54480F566
:105BC700B58006E5B5547FF5B5A233920A9006D79E
:105BD700E06003122BDEA234300B01B3500FA23466
:105BE700B34004D2878002C287A234920B9006DBAF
:105BF700E06003122CBAA235300C01B3500FA23566
:105C0700B34004D2908002C290A235920C900061FA
:105C1700E0C3945A5010E56FB40909900061E0049D
:105C2700F0756F00803BE56FB40903756F0075551C
:105C370000755400758D00758B00756400900060C9
:105C4700E0C3942A5008900060E004F08006742AAC
:105C5700900060F0900060E0B42A06E5B554FEF5C8
:105C6700B5900061E0D394014007E56AC3944140D1
:0F5C7700028009740E90003FF0123F900248B176
:105D16000000010001400160018001A001C001E016
:105D260002000300039603B603D603F4040005003D
:105D36000512052405360548055A056C057E0590AD
:105D460005A805C005DE0600061406280646066EEA
:105D560006AE05CF00FF013F015F017F019F01BF36
:105D660001DF01FF02FF039503B503D503F303FF2C
:105D760004FF05110523053505470559056B057D06
:105D8600058F05A705BF05CE05F1061306270645AF
:105D9600066D06AD06ED05DD0FAA0FA50F9F0F9A3E
:105DA6000F940F8D0F870F800F780F710F680F609C
:105DB6000F570F4E0F450F3B0F300F250F1A0F0EC3
:105DC6000F020EF50EE80EDB0ECC0EBE0EAE0E9FCB
:105DD6000E8E0E7D0E6C0E5A0E470E340E200E0CD5
:105DE6000DF70DE20DCB0DB50D9D0D850D6D0D5409
:105DF6000D3A0D200D050CE90CCE0CB10C940C7669
:105E06000C580C3A0C1B0BFB0BDB0BBB0B9A0B79E0
:105E16000B570B350B130AF10ACE0AAB0A870A6435
:105E26000A400A1C09F809D409B0098C0967094314
:105E3600091F08FB08D608B2088E086A0846082318
:105E460007FF07DC07B9079607730751072F070DEA
:105E560006EC06CA06AA068906690649062A060A3D
:105E660005EC05CD05B0059205750558053C0520E0
:105E7600050504EA04CF04B5049C048204690451B0
:105E860004390422040B03F403DE03C803B2039DA2
:105E9600038903750361034D033B032803160304BB
:105EA60002F202E102D102C002B002A00291028215
:105EB6000273026502570249023C022F02220216B1
:105EC600020901FD01F201E601DB01D001C601BBB9
:105ED60001B101A7019D0194018B01820179017035
:105EE6000168016001580150014801410139013240
:105EF600012B0125011E01180111010B010500FFEF
:105F060000FA0FA60FA00F990F920F8B0F840F7C2C
:105F16000F740F6B0F620F580F4E0F430F380F2C75
:105F26000F1F0F120F050EF70EE80ED80EC80EB78C
:105F36000EA50E930E800E6C0E580E420E2C0E15EC
:105F46000DFD0DE40DCB0DB10D950D790D5D0D3FDC
:105F56000D200D010CE10CC00C9E0C7C0C590C356F
:105F66000C100BEA0BC40B9E0B760B4F0B260AFD8F
:105F76000AD40AAA0A800A550A2A09FF09D409A8D6
:105F8600097C0950092508F908CD08A10875084AB1
:105F9600081E07F307C8079D07730749072006F77A
:105FA60006CE06A6067E06570630060A05E405BF97
:105FB600059B057705540532051004EF04CE04AEA3
:105FC600048F047104530435041903FD03E203C767
:105FD60003AD0394037B0363034B0334031E0308DF
:105FE60002F302DE02CA02B602A30291027F026D2A
:105FF600025C024C023C022C021D020E020001F25F
:1060060001E401D701CA01BE01B101A6019A018FBF
:106016000185017A01700166015D0153014A014162
:10602600013901310129012101190112010B010474
:1060360000FD00F700F000EA00E400DE00D900D31E
:1060460000CE00C900C400BF00BA00B500B100AD63
:1060560000A800A400A0009C009900950091008E65
:0C606600008A008700840081007E007B1F
:10009E007547009007B4E4F0A3F075310075300099
:1000AE00754D00754E00C237D23874FE9007B6F803
:1000BE00E4F0E8A3F074FE9007B8F8E4F0E8A3F0DB
:1000CE0074FE9007C2F0745A9007C3F0745A9007EA
:1000DE00C4F0D239C22BC23BC23622750B00750A50
:1000EE0000AE0AAF0BAC08AD09EDC39FEC9E4016F7
:1000FE0074FF12641E75CF01780B740126F650043E
:10010E0018E436F650DB2290003BE0B4AA1C9007B0
:10011E0070E0B43C159007B0E0FEA3E0FFEF4E6038
:10012E0009741EBE0004D39F5003020243755D0086
:10013E00755C0075F8099007B0E0FEA3E0FF740748
:10014E006F4E6006740E6F4E7006743A900770F024
:10015E009007B0E0FEA3E0FF7408BE001ED39F40E0
:10016E001A7E017F089007B0E0FCA3E0FD1DBDFFE5
:10017E00011C1200038E5A8F5B801F9007B0E0FEA9
:10018E00A3E0FF74081264828F048E057E017F083F
:10019E00CDCCCD1200038E5A8F5BAE5CAF5D740C6E
:1001AE00D39F74019E500302023EA2F9B3407EE536
:1001BE005D455C700375A382AE5CAF5D74016F4EDE
:1001CE00700375A300AE5CAF5D74026F4E700D9040
:1001DE0007B1E075F002A4FDACF08DA3AE5CAF5D8F
:1001EE0074036F4E700375A300AE5CAF5D7403BEF7
:1001FE0000039F5013AC5AAD5BED2FFFEC3EFE900B
:10020E00006C126465E0F5A3AE5CAF5DEFB40B0954
:10021E00EEB40105741412641EAE5CAF5DEFB40B48
:10022E0007EEB4010375F80D785C1264920201A812
:10023E0090003BE4F022755D00755C0075F8099046
:10024E0007B0E0FEA3E0FF7408BE001ED39F401A65
:10025E007E017F089007B0E0FCA3E0FD1DBDFF010D
:10026E001C1200038E5A8F5B801F9007B0E0FEA316
:10027E00E0FF74081264828F048E057E017F08CD24
:10028E00CCCD1200038E5A8F5BAE5CAF5D7411D372
:10029E009F74019E5003020374A2F9B3500302032C
:1002AE0071E55D455C700375A3D2AE5CAF5D740104
:1002BE006F4E700375A300AE5CAF5D74026F4E702F
:1002CE000D9007B1E075F002A4FDACF08DA3AE5C0D
:1002DE00AF5D74036F4E700375A300AE5CAF5D74BB
:1002EE00046F4E700375A300AE5CAF5D74056F4E68
:1002FE00700375A300AE5CAF5D74066F4E70037530
:10030E00A300AE5CAF5D74076F4E700375A300AEB5
:10031E005CAF5D74086F4E700375A300AE5CAF5D8D
:10032E007408BE00039F5016AC5AAD5BED2FFFEC68
:10033E003EFE900067126465E5A3F075A300AE5C07
:10034E00AF5DEFB41009EEB40105741412641EAE65
:10035E005CAF5DEFB41007EEB4010375F80D785C79
:10036E0012649202029722755D00755C0075F809A1
:10037E00AE5CAF5D7417BE0004D39F500302044DF4
:10038E00A2F9B3500302044AE55D455C700375A300
:10039E00D2AE5CAF5D74016F4E700375A300AE5CA0
:1003AE00AF5D74026F4E700D9007B1E075F002A450
:1003BE00FDACF08DA3AE5CAF5D74036F4E70037534
:1003CE00A300AE5CAF5D74046F4E700375A300AEF8
:1003DE005CAF5D74056F4E700375A300AE5CAF5DD0
:1003EE0074066F4E700375A300AE5CAF5D74076F3D
:1003FE004E700375A300AE5CAF5D74086F4E700354
:10040E0075A300AE5CAF5D7408BE00039F500C90E8
:10041E000049126465E5A3F075A300AE5CAF5D7490
:10042E00166F4E7005741412641EAE5CAF5D7416BA
:10043E006F4E700375F80D785C12649202037E2283
:10044E0090003BE0B4AB0280030204E8755D0075DA
:10045E005C0075F809AE5CAF5D7412BE007CD39F74
:10046E004078A2F9B34070E55D455C700375A382D8
:10047E00AE5CAF5D74016F4E700375A300AE5CAFE2
:10048E005D74026F4E700D9007B1E075F002A4FD21
:10049E00ACF08DA3AE5CAF5D74036F4E700375A3AD
:1004AE0000AE5CAF5D7403BE00039F500990004E1A
:1004BE00126465E0F5A3AE5CAF5D74116F4E70050E
:1004CE00741412641EAE5CAF5D74116F4E700375C2
:1004DE00F80D785C126492020463229007BFE4F078
:1004EE0074649007B0F8E4F0E8A3F012037574C8D2
:1004FE009007B0F8E4F0E8A3F074FF900049F074B0
:10050E00FF90004AF074FF90004BF074009000438F
:10051E00F074FF90004CF0740090004EF074019057
:10052E00004FF0900055E0B4371A900052E0900062
:10053E0049F0900053E090004AF0900054E0900093
:10054E004BF080469007BF7401F074659007B0F8C9
:10055E00E4F0E8A3F012037574C89007B0F8E4F065
:10056E00E8A3F0900055E0B4371A900052E09000E6
:10057E0049F0900053E090004AF0900054E0900053
:10058E004BF0800674029007BFF09007C0E4F07441
:10059E00669007B0F8E4F0E8A3F012037574C89003
:1005AE0007B0F8E4F0E8A3F0900054E0B4371290EE
:1005BE000052E0900043F0900053E090004CF08029
:1005CE00769007C07401F074679007B0F8E4F0E815
:1005DE00A3F012037574C89007B0F8E4F0E8A3F026
:1005EE00900054E0B43712900052E0900043F09027
:1005FE000053E090004CF0803E74029007C0F074FF
:10060E00689007B0F8E4F0E8A3F012037574C89090
:10061E0007B0F8E4F0E8A3F0900054E0B43712907D
:10062E000052E0900043F0900053E090004CF080B8
:10063E000674039007C0F022E54E64046006E59947
:10064E0064FF60028031A2374004D2378027E54E26
:10065E00600874E6254E90003FF0E54D600874F09A
:10066E00254D90003FF0E54EB4010280FE754E0020
:10067E00754D00C2378002C237E54E90384AF828D1
:10068E002873754E00E599B4FF03754D01E599B4D5
:10069E00FE03754D02E599B4FD03754D03E599B45E
:1006AE00FC03754D04E599B4FA03754D05E599B44F
:1006BE00FB06754E01123F90E599B4F906754E048E
:1006CE00123F90E599D394E54007E599C394F04025
:1006DE0002801685994F754E027E017F00E54FC34D
:1006EE0094E612643E8E328F339007B4E4F0A3F09A
:1006FE00E599D394C44007E599C394E64002802857
:10070E0085994F754E0374E5C3954FF533753200D9
:10071E00AE32AF33905D1612640DE493F87401930C
:10072E009007B4C8F0A3C8F0D299020C56900052AC
:10073E00E07005A229B3400280429007B4E0FEA308
:10074E00E0FF74FFBE00039F5009EFC39446EE9482
:10075E000640119007B4E0FEA3E0FFEFD3946DEED8
:10076E00940640139007B4E0FEA3E0FF90007012D1
:10077E006465E599F0800385997480119007B4E063
:10078E00FEA3E0FF900070126465E599F09007B447
:10079E0012644C9007B4E0FEA3E0FFEFB40106EE46
:1007AE00B4070280030209FD900770E0B43C02809A
:1007BE00030209FDA22950030208E8C29C900052D0
:1007CE00E090010EF0900053E090007DF090005408
:1007DE00E090009DF0900055E09000C6F09000561D
:1007EE00E0900072F0900057E09000B8F090005842
:1007FE00E09000D6F0900059E09000AAF090005AD8
:10080E00E09000C8F090005BE09000F8F090005C83
:10081E00E090015CF090005DE090015DF090005E74
:10082E00E090015EF0123B6E900064E09000DFF00D
:10083E00900065E0900096F0900066E0900097F0D2
:10084E0074639007B0F8E4F0E8A3F074AB90003B4B
:10085E00F012044E90003BE4F07464F50975080044
:10086E001200E9A21E4039757301E573D394075047
:10087E002DE5739007B0F8E4F0E8A3F074AA9000A9
:10088E003BF0120115E573C39407500A7464F50921
:10089E007508001200E97873740126F650CC803783
:1008AE00757308E573D3940E502DE5739007B0F869
:1008BE00E4F0E8A3F074AA90003BF0120115E57382
:1008CE00C3940E500A7464F5097508001200E97895
:1008DE0073740126F650CC0209E7C29C90010EE01B
:1008EE00900052F090007DE0900053F090009DE05B
:1008FE00900054F09000C6E0900055F0900072E029
:10090E00900056F09000B8E0900057F09000D6E0BE
:10091E00900058F09000AAE0900059F09000C8E0C6
:10092E0090005AF09000F8E090005BF07400900098
:10093E005CF0740090005DF0740090005EF07463E3
:10094E009007B0F8E4F0E8A3F074AB90003BF0121F
:10095E00044E90003BE4F07464F509750800120033
:10096E00E9757301E573D394075026E5739007B0CC
:10097E00F8E4F0E8A3F074AA90003BF012011574AD
:10098E0064F5097508001200E97873740126F650B3
:10099E00D3D29C7599FB743C900770F0757308E583
:1009AE0073D3940E5026E5739007B0F8E4F0E8A3E5
:1009BE00F074AA90003BF01201157464F5097508E5
:1009CE00001200E97873740126F650D374C89007AC
:1009DE00B0F8E4F0E8A3F080FE74C89007B0F8E435
:1009EE00F0E8A3F0D29C754E00754D007599FB0290
:1009FE000C569007B4E0FEA3E0FFEF4E700685990B
:100A0E00317530009007B4E0FEA3E0FF74016F4E25
:100A1E00701BAC30AD31AA32AB33ED2BFBEC3AFA96
:100A2E008A068B07900070126465E599F09007B402
:100A3E0012644C9007B4E0FEA3E0FF74026F4E7098
:100A4E0021AC30AD3174566D4C7006E54F64E660E6
:100A5E00028003123F90123B6E854F99754E0075C2
:100A6E004D00020C569007B4E0FEA3E0FF9000701C
:100A7E00126465E599F09007B412644C9007B4E0E7
:100A8E00FEA3E0FFAC32AD338F028E038C068D07D2
:100A9E00905D5A12640DE493F9740193FEEAD39EAD
:100AAE00EB994009854F99754E00754D00020C5615
:100ABE009007B4E0FEA3E0FF900070126465E59924
:100ACE00F09007B412644C9007B4E0FEA3E0FFEF81
:100ADE00B40006EEB401028003020C5690004BE007
:100AEE00D394C7400B90004BE0C394C8F550801AC6
:100AFE0090004BE0D39463400B90004BE0C39464A2
:100B0E00F550800690004BE0F550E55075F002A4CC
:100B1E00FFAEF08F73EF900070126470EFFCE0FD8B
:100B2E00EC900073126470EDFCE0FDEC2DB55002FC
:100B3E008003020C470FEF900070126470E573FF94
:100B4E00E0FCEF900074126470ECFFE0FCEFC39CCD
:100B5E00B550028003020C47E57390007212647068
:100B6E00E573FFE0FCEF900075126470ECFFE0FCA3
:100B7E00EF2CB550028003020C47E57390007612FD
:100B8E006470E0C39550900052F0E57390007712B8
:100B9E006470E0C39550900053F0E57390007812A6
:100BAE006470E0C39550900054F07400900055F0BE
:100BBE0074FF900056F0E57390007A126470E0C3F3
:100BCE009550900057F0E57390007B126470E0C36F
:100BDE009550900058F0E57390007C126470E0C35D
:100BEE009550900059F0E573900079126470E0C34F
:100BFE0095509007B0F8E4F0E8A3F074AB90003B8A
:100C0E00F012044E7464F5097508001200E990079D
:100C1E00B012644C12044E7464F50975080012008B
:100C2E00E99007B012644C12044E7599F97464F58C
:100C3E00097508001200E980FE7599FF7464F509C4
:080C4E007508001200E980FEA8
:0F384A0002069002073B020A00020A73020ABE3E
:100C560022E54D903859F8282873020D699007B49B
:100C6600E0FEA3E0FF900041126465E0F59990076D
:100C7600B412644C9007B4E0FEA3E0FF74116F4E0B
:100C86007003754D00020D69856E99020D69900716
:100C9600B4E0FEA3E0FF900070126465E0F599EF02
:100CA600B40107EEB40703754D009007B412644C07
:070CB600020D699007B5E093
:0F385900020C60020C63020C8E020C94020CB97C
:100CBD00903A0CF8282873855399020D5E855F993B
:100CCD00020D5E856199020D5E856599020D5E8549
:100CDD006799807D85689980788569998073856A23
:100CED0099806E900016E0F5998066A238B34007A2
:100CFD007599FAC2388041A228B3400575990F80C5
:100D0D00359007BFE0600A9007BFE024DCF59980BD
:100D1D00169007C0E0600A9007C0E024DEF59980C8
:100D2D000690003FE0F59990003FE4F09007BFE496
:100D3D00F09007C0E4F0C2288017856B998012856A
:100D4D006699800D856C9980087599FC8003754DA9
:010D5D000095
:103A0C00020CC4020CCA020CD0020CD6020CDC0252
:103A1C000CE1020CE6020CEB020CF0020CF8020DAD
:0D3A2C0047020D4C020D51020D56020D5BBC
:0B0D5E009007B412644C8003123A3975
:03386800020D66E8
:100D690022E537255BFFAE5A50010E9000701264E0
:100D790065E0F538E537255BFFAE5A50010E0FBF28
:100D890000010E900070126465E0F539853F3BE57E
:100D990038B539058538378041E539D39538401D4F
:100DA900E539C39538853AF0A4FFAEF0E53B8E04EA
:100DB9008F05FF12642EED2538F537801DE538C300
:100DC9009539853AF0A4FFAEF0E53B8E048F05FF17
:100DD90012642EEDF4042538F53722E539D3953818
:100DE900401DE539C39538853AF0A4FFAEF0E53BDF
:100DF9008E048F05FF12642EED2538F537801DE529
:100E090038C39539853AF0A4FFAEF0E53B8E048FDF
:100E190005FF12642EEDF4042538F537229000768B
:100E2900E0B40170E56775F00A84FF7E008F37E54D
:100E39006775F00A84ADF07C008D3A753F0A755AE2
:100E490005755B24E537C394115005120D6A8006B8
:100E59009005A5E0F537E537900069F0E56775F08D
:100E69000A84FF7E008F37E56775F00A84ADF07C50
:100E7900008D3A753F0A755A05755B5AE537C39473
:100E8900115005120D6A80069005DBE0F537E5374C
:100E990090000EF022900076E0B4016AE56775F0E3
:100EA9000A84FF7E008F37E56775F00A84ADF07C10
:100EB900008D3A753F0A755A05755B36E537C39457
:100EC900115005120D6A80069005B7E0F537853790
:100ED9004BE56775F00A84FF7E008F37E56775F08B
:100EE9000A84ADF07C008D3A753F0A755A05755B29
:100EF90048E537C394115005120D6A80069005C95B
:100F0900E0F53785374C22E55F75F00484FF7E00F4
:100F19008F37E55F75F00484ADF07C008D3A753F3D
:100F290004755A01755B00E537C3943F5005120DEE
:100F39006A80069001AFE0F537853729752800905A
:100F4900003EE075F020A4FFAEF09000C1E08E04F1
:100F59008F05FF12642E8D379000A9E0D3955F505D
:100F6900030210169000CDE0D3955F4010ED90017B
:100F7900B0126470E0F52B752A00021013900098E6
:100F8900E0D3955F4043E5379001B0126470E0F516
:100F990038E5379001D0126470E0F5399000CDE062
:100FA900F404255FF53A900098E0FE9000CDE0F456
:100FB900042EF53BE538B539058538378003120D20
:100FC900E485372B752A008041E5379001D01264FA
:100FD90070E0F538E5379001F0126470E0F539906A
:100FE9000098E0F404255FF53A9000A9E0FE90002E
:100FF90098E0F4042EF53BE538B539058538378096
:1010090003120DE485372B752A000210BD9000D01C
:10101900E0D3955F5011E537900230126470E0F526
:101029002B752A000210BD900099E0D3955F5043BB
:10103900E537900210126470E0F538E53790023018
:10104900126470E0F539900099E0F404255FF53AEF
:101059009000D0E0FE900099E0F4042EF53BE538CD
:10106900B539058538378003120DE485372B752A84
:10107900008041E5379001F0126470E0F538E537FA
:10108900900210126470E0F5399000A9E0F404258B
:101099005FF53A900099E0FE9000A9E0F4042EF57E
:1010A9003BE538B539058538378003120DE48537B6
:1010B9002B752A00229000E1E0F53C753F11755A25
:1010C90002755B00AE52AF53E53C75F00FA4FDAC61
:1010D900F0EDD39FEC9E4021E53C8E048F05FF1275
:1010E900642EED75F010A4FFAEF0E55F75F0118484
:1010F900FD7C00ED2FF53D800EE55F75F01184FF55
:101109007E00EF24F0F53D853D37E55F75F01184EC
:10111900AFF07E008F3A120D6A85373EAE52AF535B
:101129009000E1E075F00FA4FDACF0EDD39FEC9ECB
:101139004028755A02755B10853D37120D6A853E48
:1011490038853739AE52AF53E53C8E048F05FF120F
:1011590064598D3A853C3B120DE485372975280081
:10116900752B64752A00229000E1E0F53C753F116A
:10117900755A02755B00AE52AF53E53C75F00FA48A
:10118900FDACF0EDD39FEC9E4021E53C8E048F052C
:10119900FF12642EED75F010A4FFAEF0E56175F055
:1011A9001184FD7C00ED2FF53D800EE56175F01190
:1011B90084FF7E00EF24F0F53D853D37E56175F04C
:1011C9001184AFF07E008F3A120D6A85373EAE5218
:1011D900AF539000E1E075F00FA4FDACF0EDD39FA3
:1011E900EC9E4028755A02755B10853D37120D6AD1
:1011F900853E38853739AE52AF53E53C8E048F05AD
:10120900FF1264598D3A853C3B120DE485372975E7
:101219002800E56B6017E56BC394FE50109000D56C
:10122900E0B402099000C3E0D3940B50028017AEDA
:1012390028AF29E56B12643E74E78E048F05FF120F
:10124900642E8C288D299000ABE0B40453E55F75BA
:10125900F00484FF7E008F37E55F75F00484ADF0FC
:101269007C008D3A753F04755A01755B00E537C3FB
:10127900943F5005120D6A80069001AFE0F537AE34
:1012890028AF29E53712643E74648E048F05FF1276
:10129900642EAE28AF29EF2DFDEE3CFC8C288D295C
:1012A900752B64752A0022900076E0B40146E56743
:1012B90075F00A84FF7E008F37E56775F00A84AD03
:1012C900F07C008D3A753F0A755A05755B00E53764
:1012D900C394115005120D6A8006900581E0F53717
:1012E900AE2AAF2BE5372FFF50010E7464126482CA
:1012F9008E2A8F2B900077E0B40146E56875F00AD5
:1013090084FF7E008F37E56875F00A84ADF07C00B4
:101319008D3A753F0A755A05755B6CE537C39411AB
:101329005005120D6A80069005EDE0F537AE2AAF3B
:101339002BE5372FFF50010E74641264828E2A8FB9
:101349002B900086E0B40249E56AC3944175F00523
:1013590084FF7E008F37E56A75F00584ADF07C0067
:101369008D3A753F05755A06755B00E537C39413C9
:101379005005120D6A8006900683E0F537AE2AAF54
:101389002BE5372FFF50010E74641264828E2A8F69
:101399002B9000C8E0B40202800302144FE55F7588
:1013A900F01584FF7E008F37E55F75F01584ADF089
:1013B9007C008D3A753F15755A03755BF4E537C3A3
:1013C900940B5005120D6A800690046FE0F537E51D
:1013D9003775F0FFA4FFAEF09000C9E08E048F05C9
:1013E900FF12642EED900062F0E56675F078A4FFB7
:1013F900AEF074FF8E048F05FF12642E8C5A8D5B3C
:1014090074028C068D071200398F37AC5AAD5B74A4
:1014190004FF1264598D3A753F04755A06755B28A5
:10142900E537C3941D5005120D6A80069006B5E094
:10143900F537AE2AAF2BE5372FFF50010E74641232
:1014490064828E2A8F2B900075E0B4025DE5617588
:10145900F064A4FFAEF074081200398E5C8F5D74DD
:10146900058E048F05FF12642E8D37AE5CAF5D7457
:10147900058E048F05FF1264598D3A753F05755A1B
:1014890005755BDEE537C394135005120D6A8006B6
:10149900900661E0F537AE2AAF2BE5372FFF5001F3
:1014A9000E74641264828E2A8F2B9000B7E0703C10
:1014B90090003EE075F00584FF7E008F3790003E76
:1014C900E075F00584ADF07C008D3A753F05755ADD
:1014D90005755BC0E537C3941D5005120D6A80067A
:1014E90090064DE0F537E53790006AF02290007ECE
:1014F900E0B401179007BBE0252BFFAE2A50010E7F
:101509009000D2E01264828E2A8F2B9000F6E0B40C
:1015190001149000F7E0A852B8000495535007E56C
:101529005FC39560400280129000A0E0252BFFAEBA
:101539002A50010E8E2A8F2B802F90007EE0B40353
:1015490016A22BB3B350109007BEE0C39405A8525E
:10155900B800069553400280109000A0E0252BFFAB
:10156900AE2A50010E8E2A8F2B900078E0B4020229
:1015790080030218F490007BE0602FE567D394465E
:10158900402890000FE0FEA3E0FF9000B6E075F060
:1015990003A4FDACF0EFD39DEE9C400E9000DAE081
:1015A900A852B80005D3955350030218F49000AB24
:1015B900E0B40302800302175885615B755A0090F5
:1015C9000082E0A852B800049553500E900083E0C1
:1015D900A85AB80005D3955B5003021755E5617504
:1015E900F002A4FFAEF074158E048F05FF12642E6D
:1015F9008C068D07900600126465FEE0FFEE9000F0
:101609007AE0FEEF8E0088F0A4FFAEF074648E04D9
:101619008F05FF12642E8C5A8D5B90003EE075F0A9
:1016290018A4FFAEF09000C1E08E048F05FF12648C
:101639002E8C068D07900618126465AE5AAF5BE0D2
:1016490012643E74648E048F05FF12642E8C5A8DC9
:101659005BE565A85AB80077D3955B4072E565C329
:10166900955BFFE4955AFE8E5A8F5B7428BE000382
:101679009F500C755B28755A00740D90003FF0AEB1
:101689005AAF5B90007BE012643E74288E048F058C
:10169900FF12642E8C5A8D5BAE28AF29740A8E0412
:1016A9008F05FF12642E8D068C07AC5AAD5BCFCE29
:1016B900CF120003740A8E048F05FF12642E8C5A10
:1016C9008D5BAE28AF2912648A8E288F29807DE52B
:1016D90065A85AB80004955B5072AE5AAF5BE565D0
:1016E9001264828E5A8F5B7428BE00039F500C755A
:1016F9005B28755A00740D90003FF0AE5AAF5B90AD
:10170900007BE012643E74288E048F05FF12642E5C
:101719008C5A8D5BAE28AF29740A8E048F05FF128F
:10172900642E8D068C07AC5AAD5BCFCECF12000369
:10173900740A8E048F05FF12642E8C5A8D5BAE28B5
:10174900AF29EF2DFDEE3CFC8C288D290218F49071
:1017590000C3E0855FF0A4FFAEF0740512643E7427
:10176900071200398E5A8F5B900082E0A852B800A8
:101779000495535012900083E075F002A4FDACF07B
:10178900EFC39DEE9C40030218F4E55F75F00B84EE
:10179900FF7E00900600126465FEE0FFEE90007A7D
:1017A900E0FEEF8E0088F0A4FFAEF074648E048F23
:1017B90005FF12642E8C5A8D5B90003EE075F0187F
:1017C900A4FFAEF09000C1E08E048F05FF12642ED5
:1017D9008C068D07900618126465AE5AAF5BE0124D
:1017E900643E74648E048F05FF12642E8C5A8D5BDF
:1017F900E565A85AB80077D3955B4072E565C3954E
:101809005BFFE4955AFE8E5A8F5B7428BE00039FD6
:10181900500C755B28755A00740D90003FF0AE5A54
:10182900AF5B90007BE012643E74288E048F05FF45
:1018390012642E8C5A8D5BAE28AF29740A8E048FE0
:1018490005FF12642E8D068C07AC5AAD5BCFCECF47
:10185900120003740A8E048F05FF12642E8C5A8DB0
:101869005BAE28AF2912648A8E288F29807DE565B1
:10187900A85AB80004955B5072AE5AAF5BE5651281
:1018890064828E5A8F5B7428BE00039F500C755B6F
:1018990028755A00740D90003FF0AE5AAF5B900066
:1018A9007BE012643E74288E048F05FF12642E8C2F
:1018B9005A8D5BAE28AF29740A8E048F05FF126416
:1018C9002E8D068C07AC5AAD5BCFCECF12000374B8
:1018D9000A8E048F05FF12642E8C5A8D5BAE28AFD9
:1018E90029EF2DFDEE3CFC8C288D29229000D6E0B5
:1018F900B4026AE55F75F00884FF7E008F37E55F03
:1019090075F00884ADF07C008D3A753F08755A0171
:10191900755BE0E537C3943F5005120D6A80069068
:10192900026FE0F53785372D752C00AE2CAF2DAC45
:101939002AAD2B12000374648E048F05FF12642EE6
:101949008C2C8D2D900073E08C068D0712643E74EB
:10195900648E048F05FF12642E8C2C8D2DAE28AF5A
:1019690029AC2AAD2B12000374648E048F05FF1273
:10197900642E8C288D29900073E08C068D071264E3
:101989003E74648E048F05FF12642E8C288D29A263
:101999000D401DAE52AF537405BE00039F5002D2D5
:1019A9000DE561D394CC4008D201741190003FF049
:1019B9009000D5E0B402089000C3E0640B60028097
:1019C90035AE28AF29E56B12643E74E78E048F05A6
:1019D900FF12642E8C288D299000D6E0B40217AE30
:1019E9002CAF2DE56B12643E74E78E048F05FF1250
:1019F900642E8C2C8D2D900095E05402601B900074
:101A09008CE0A852B80012D39553400DA20DB3B380
:101A19005007E561C3949A40028028AE34AF3590EF
:101A2900008AE075F002A4FDACF0EF2DFDEE3CFC60
:101A390074022DFD50010CE561BC0007D39D4003E4
:101A4900754301856135753400E5437003021B3820
:101A59009000E8E0C395435003021B2A9000F8E088
:101A6900C394025076E56775F00A84FF7E009005FD
:101A790070126465E0F55B755A00AE5AAF5B900071
:101A89008BE012643E74648E048F05FF12642E8C01
:101A99005C8D5D9000E8E004C395438C068D0712C8
:101AA900643E9000E8E08E048F05FF12642E8C5C82
:101AB9008D5DAE28AF29EF2DFDEE3CFC8C288D29DC
:101AC9009000D6E0B40212AE2CAF2DAA5CAB5DEF4C
:101AD9002BFBEE3AFA8A2C8B2D80469000E8E00425
:101AE900C39543854BF0A4FFAEF09000E8E08E0467
:101AF9008F05FF12642E8C5C8D5DAE28AF29EF2D0A
:101B0900FDEE3CFC8C288D299000D6E0B40212AE83
:101B19002CAF2DAA5CAB5DEF2BFBEE3AFA8A2C8B2E
:101B29002D05439000E8E0C39543500375430090A9
:101B39000095E05401601B900089E0A852B800129A
:101B4900D39553400DA20DB3B35007E55FC394CCB1
:101B590040028025900087E075F003A4FFAEF0E510
:101B6900402FFF50010E74032FFF50010EE55FBE99
:101B79000007D39F4003754401855F40E544700326
:101B8900021C6B9000E9E0C395445003021C5D9070
:101B990000F8E0C394025076E56775F00A84FF7E89
:101BA90000900570126465E0F55B755A00AE5AAF96
:101BB9005B900088E012643E74648E048F05FF1206
:101BC900642E8C5C8D5D9000E9E004C395448C061D
:101BD9008D0712643E9000E9E08E048F05FF1264C0
:101BE9002E8C5C8D5DAE28AF29EF2DFDEE3CFC8C73
:101BF900288D299000D6E0B40212AE2CAF2DAA5C34
:101C0900AB5DEF2BFBEE3AFA8A2C8B2D80469000C8
:101C1900E9E004C39544854CF0A4FFAEF09000E9D7
:101C2900E08E048F05FF12642E8C5C8D5DAE28AFAB
:101C390029EF2DFDEE3CFC8C288D299000D6E0B4CF
:101C49000212AE2CAF2DAA5CAB5DEF2BFBEE3AFA7C
:101C59008A2C8B2D05449000E9E0C3954450037507
:101C690044009000EBE02529FFAE2850010E8E2894
:101C79008F2990009AE0A828B80004952950099066
:101C8900009AE0F5297528009000D6E0B4020D907D
:101C9900009AE0A82CB80006952D40028009900012
:101CA9009AE0F52D752C00229000D6E0B40102804F
:101CB90003021DBCA20DB35003021DBA9000A1E09E
:101CC900B40168AE28AF29AC52AD53120003743C7D
:101CD9008E048F05FF12642E9000B1E0BC00109DA8
:101CE900400D9000B3E0A828B8000495295002D20D
:101CF90002AE28AF29AC52AD53120003743C8E04D6
:101D09008F05FF12642E9000B1E0C3940ABC001540
:101D1900D39D40119000B3E0C39405A828B80005ED
:101D2900D3952950028002C2028068AE28AF29AC3F
:101D390052AD5312000374788E048F05FF12642E7E
:101D49009000B1E0BC00109D400D9000B3E0A828C0
:101D5900B8000495295004D2028038AE28AF29ACC6
:101D690052AD5312000374788E048F05FF12642E4E
:101D79009000B1E0C3940ABC0015D39D40119000B6
:101D8900B3E0C39405A828B80005D395295002806B
:101D990002C202A202B34019AE28AF299000B2E0F4
:101DA90012643E74648E048F05FF12642E8C288D94
:101DB900298002C202A200B34006A201B3B35009AE
:101DC900900015E4F0A3F08024AE28AF297400D365
:101DD9009F74019E400C900015E528F0A3E529F0B9
:101DE900800B74FF900015F8E4F0E8A3F09000B8B8
:101DF900E0D39402400C9000A3E07006A20DB3B3A7
:101E09004002801AAE28AF29740212643E8E288FD0
:101E190029AE2CAF2D740212643E8E2C8F2D9000AA
:101E2900A1E0B4011AAE28AF29740212643E8E28CB
:101E39008F29AE2CAF2D740212643E8E2C8F2DAEDD
:101E490028AF29745E12643E740A8E048F05FF124E
:101E5900642E8C288D299000D6E0B40217AE2CAFE1
:101E69002D745E12643E740A8E048F05FF12642E6F
:101E79008C2C8D2DAE28AF297402BE000AD39F4049
:101E890006752902752800AE2CAF2D7402BE000A12
:101E9900D39F4006752D02752C00900013E528F09C
:101EA900A3E529F02290003EE0900370126470E0EF
:101EB900F54175426490003EE0FE9000ACE0D39E8F
:101EC9004037E55F75F00884FF7E008F37E55F7561
:101ED900F00884ADF07C008D3A753F08755A03759A
:101EE9005B96E537C3941F5005120D6A800690046E
:101EF90025E0F5378537428035E55F75F00884FFC1
:101F09007E008F37E55F75F00884ADF07C008D3A6F
:101F1900753F08755A03755BB6E537C3941F5005BD
:101F2900120D6A8006900445E0F537853742229004
:101F390000E2E0F53C753F11755A04755B00AE523D
:101F4900AF53E53C75F00FA4FDACF0EDD39FEC9ECB
:101F59004021E53C8E048F05FF12642EED75F010CB
:101F6900A4FFAEF0E55F75F01184FD7C00ED2FF55F
:101F79003D800EE55F75F01184FF7E00EF24F0F5DA
:101F89003D853D37E55F75F01184AFF07E008F3AEE
:101F9900120D6A85373EAE52AF539000E2E075F0FC
:101FA9000FA4FDACF0EDD39FEC9E4028755A047543
:101FB9005B10853D37120D6A853E38853739AE523B
:101FC900AF53E53C8E048F05FF1264598D3A853C69
:101FD9003B120DE4853741754264229000E2E0F539
:101FE9003C753F11755A04755B00AE52AF53E53C21
:101FF90075F00FA4FDACF0EDD39FEC9E4021E53CBC
:102009008E048F05FF12642EED75F010A4FFAEF05B
:10201900E56175F01184FD7C00ED2FF53D800EE53D
:102029006175F01184FF7E00EF24F0F53D853D37A1
:10203900E56175F01184AFF07E008F3A120D6A8563
:10204900373EAE52AF539000E2E075F00FA4FDACFD
:10205900F0EDD39FEC9E4028755A04755B10853DC1
:1020690037120D6A853E38853739AE52AF53E53C94
:102079008E048F05FF1264598D3A853C3B120DE49D
:102089008537417542649000ABE0B4047990003E15
:10209900E0FE9000ACE0D39E4037E55F75F0088420
:1020A900FF7E008F37E55F75F00884ADF07C008D09
:1020B9003A753F08755A03755B96E537C3941F5007
:1020C90005120D6A8006900425E0F53785374280B0
:1020D90035E55F75F00884FF7E008F37E55F75F0A1
:1020E9000884ADF07C008D3A753F08755A03755B1D
:1020F900B6E537C3941F5005120D6A800690044552
:10210900E0F53785374222900076E0B4013BE56778
:1021190075F00A84FF7E008F37E56775F00A84AD94
:10212900F07C008D3A753F0A755A05755B12E537E3
:10213900C394115005120D6A8006900593E0F53796
:10214900E5422537C39464F542900077E0B4013B3A
:10215900E56875F00A84FF7E008F37E56875F00A37
:1021690084ADF07C008D3A753F0A755A05755B7E22
:10217900E537C394115005120D6A80069005FFE0FA
:10218900F537E5422537C39464F542E5412542F523
:102199003690007EE0B402109007BAE02536FE9032
:1021A90000D2E0F4042EF5369000D5E0D394014036
:1021B90040E56BC394E7501D74E7C3956BFE900728
:1021C900BCE08E00F5F0E884FF7E008F37E5362508
:1021D90037F536801CE56BC394E7FE9007BCE08EAB
:1021E90000F5F0E884FF7E008F37E536C39537F5B3
:1021F90036A20D4006E5412464F536E536D39464EC
:102209004009E536C39464F53680037536009000BD
:10221900AEE0C3953650069000AEE0F53622D20006
:10222900900068E0A852B8000495535041900068A6
:10223900E0A852B800049553500375360F90006812
:10224900E004A852B800049553500375360A90006B
:1022590068E02402A852B800049553500575360564
:10226900C200900068E06006740990003FF0C23B2C
:102279007E017F009000B4E012643E9000C3E08EBE
:10228900048F05FF12642EE55FBC0017D39D401330
:102299009000BDE0B40204D23B8002C200740A90EF
:1022A900003FF09000B5E0C3956750159000C7E076
:1022B900A852B8000495535002C200740B90003F15
:1022C900F0E567C39464501D90010DE0600D900125
:1022D9000DE0A852B80006955340028008C2007468
:1022E9000B90003FF0A20040037536059000F6E020
:1022F900B401149000F7E0A852B8000495535007B0
:10230900E55FC395604002800890009FE0F5368044
:102319003A90007EE0B40306A22BB3B34002802BAF
:102329009007BEE0C39405A852B800049553500C19
:1023390090009FE0F536740C90003FF09007BEE0E6
:10234900A852B8000495535002C20085366C90001B
:1023590070E02536FE90003EE075F01E84FC7F009B
:10236900EE2CF5362290003EE075F00584FF7E00E4
:102379008F3790003EE075F00584ADF07C008D3A12
:10238900753F05755A03755BD69000C1E01475F069
:102399000584FF7E00E537BE00039F5005120D6AD4
:1023A900800BE537900446126470E0F537E5379005
:1023B90007BDF09007BDE0FE9000B0E0C39E500855
:1023C9009000B0E09007BDF022E56775F00A84FF40
:1023D9007E00900570126465E0F546E546D3946485
:1023E9004010E546C3946475F00F84FF7E008F4664
:1023F9008003754600900093E02546F5462290003B
:10240900ABE0C3940350269007AAE0FEA3E0FF7453
:1024190004120039E55F12643E740F8E048F05FFC4
:1024290012642E9007A8ECF0A3EDF080249007AA7F
:10243900E0FEA3E0FF7404120039E56112643E7402
:102449000F8E048F05FF12642E9007A8ECF0A3ED00
:10245900F0900086E0B40262E56AC3944175F00524
:1024690084FF7E008F37E56A75F00584ADF07C0046
:102479008D3A753F05755A06755B14E537C3941790
:102489005005120D6A8006900697E0F5379007A867
:10249900E0FEA3E0FF740A8E048F05FF12642EE5A7
:1024A900378C068D0712643E740A8E048F05FF125D
:1024B900642E9007A8ECF0A3EDF09007A8E0FEA326
:1024C900E0FF9007AEE0FCA3E0FDEDD39FEC9E405A
:1024D9000F9007AEE0F8A3E09007A8C8F0A3C8F0F2
:1024E900229006B7E090386BF8282873804C855302
:1024F9007380479000C3E0855FF0A4FFAEF07408D5
:102509001200398F738033856173802E85677380DC
:10251900298568738024856973801F856A73801A89
:10252900856B7380158566738010856573800B854F
:0A2539006C738006900016E0F57345
:10386B000224F50224F70224FC022510022515027E
:10387B00251A02251F02252402252902252E0225A1
:07388B003302253802253D40
:102543009006B8E0FE9006B9E0D39E404B9006B7E4
:10255300E0B404189006B9E0C395735002D22C90EE
:1025630006B8E0D395734002C22C802A9006B8E0E7
:10257300C3957350099006B9E0D395735002800256
:10258300D22C9006B8E0D3957350099006B9E0C3F6
:1025930095735002C22C802A9006B8E0D3957340FD
:1025A300099006B9E0C3957340028002C22C9006DD
:1025B300B8E0C3957340099006B9E0D39573400220
:1025C300D22C229006BBE0903892F8282873804CD6
:1025D30085537380479000C3E0855FF0A4FFAEF09E
:1025E30074081200398F738033856173802E856779
:1025F3007380298568738024856973801F856A7356
:10260300801A856B7380158566738010856573806A
:0C2613000B856C738006900016E0F573D8
:103892000225D10225D30225D80225EC0225F10208
:1038A20025F60225FB02260002260502260A02262A
:0738B2000F02261402261983
:10261F009006BCE0FE9006BDE0D39E405F9006BBE7
:10262F00E0B404189006BDE0C395735002D22D900C
:10263F0006BCE0D395734002C22D803E9006BCE0ED
:10264F00C3957350099006BDE0D395735002800275
:10265F00D22D9006BCE0D3957350099006BDE0C310
:10266F0095735002C22D9006BBE0B401099000CFC4
:10267F00E0D3956150028002C22D802A9006BCE003
:10268F00D3957340099006BDE0C395734002800255
:10269F00C22D9006BCE0C3957340099006BDE0D3F0
:1026AF0095734002D22D229006BFE09038B9F828DA
:1026BF002873804C85537380479000C3E0855FF08B
:1026CF00A4FFAEF074081200398F738033856173E5
:1026DF00802E856773802985687380248569738050
:1026EF001F856A73801A856B7380158566738010DA
:1026FF00856573800B856C738006900016E0F5730B
:1038B9000226C10226C30226C80226DC0226E1022C
:1038C90026E60226EB0226F00226F50226FA022651
:0738D900FF0227040227098A
:10270F009006C0E0FE9006C1E0D39E404B9006BFFE
:10271F00E0B404189006C1E0C395735002D22E9016
:10272F0006C0E0D395734002C22E802A9006C0E007
:10273F00C3957350099006C1E0D395735002800280
:10274F00D22E9006C0E0D3957350099006C1E0C316
:10275F0095735002C22E802A9006C0E0D395734025
:10276F00099006C1E0C3957340028002C22E900605
:10277F00C0E0C3957340099006C1E0D39573400242
:10278F00D22E229006C3E09038E0F8282873804CB0
:10279F0085537380479000C3E0855FF0A4FFAEF0D0
:1027AF0074081200398F738033856173802E8567AB
:1027BF007380298568738024856973801F856A7388
:1027CF00801A856B7380158566738010856573809D
:0C27DF000B856C738006900016E0F5730B
:1038E00002279D02279F0227A40227B80227BD02B4
:1038F00027C20227C70227CC0227D10227D60227D8
:07390000DB0227E00227E5CE
:1027EB009006C4E0FE9006C5E0D39E404B9006C316
:1027FB00E0B404189006C5E0C395735002D22F9035
:10280B0006C4E0D395734002C22F802A9006C4E021
:10281B00C3957350099006C5E0D39573500280029F
:10282B00D22F9006C4E0D3957350099006C5E0C330
:10283B0095735002C22F802A9006C4E0D395734043
:10284B00099006C5E0C3957340028002C22F900623
:10285B00C4E0C3957340099006C5E0D3957340025D
:10286B00D22F229006C7E0903907F8282873804CA6
:10287B0085537380479000C3E0855FF0A4FFAEF0F3
:10288B0074081200398F738033856173802E8567CE
:10289B007380298568738024856973801F856A73AB
:1028AB00801A856B738015856673801085657380C0
:0C28BB000B856C738006900016E0F5732E
:1039070002287902287B022880022894022899023B
:10391700289E0228A30228A80228AD0228B202285E
:07392700B70228BC0228C111
:1028C7009006C8E0FE9006C9E0D39E404B9006C72D
:1028D700E0B404189006C9E0C395735002D2309053
:1028E70006C8E0D395734002C230802A9006C8E03C
:1028F700C3957350099006C9E0D3957350028002BF
:10290700D2309006C8E0D3957350099006C9E0C34A
:1029170095735002C230802A9006C8E0D395734061
:10292700099006C9E0C3957340028002C230900641
:10293700C8E0C3957340099006C9E0D39573400278
:10294700D230229006CBE090392EF8282873804C9D
:1029570085537380479000C3E0855FF0A4FFAEF016
:1029670074081200398F738033856173802E8567F1
:102977007380298568738024856973801F856A73CE
:10298700801A856B738015856673801085657380E3
:0C2997000B856C738006900016E0F57351
:10392E0002295502295702295C02297002297502C3
:10393E00297A02297F02298402298902298E0229E5
:07394E009302299802299D54
:1029A3009006CCE0FE9006CDE0D39E404B9006CB44
:1029B300E0B404189006CDE0C395735002D2319071
:1029C30006CCE0D395734002C231802A9006CCE056
:1029D300C3957350099006CDE0D3957350028002DE
:1029E300D2319006CCE0D3957350099006CDE0C365
:1029F30095735002C231802A9006CCE0D395734080
:102A0300099006CDE0C3957340028002C23190065F
:102A1300CCE0C3957340099006CDE0D39573400293
:102A2300D231229006CFE0903955F8282873804C94
:102A330085537380479000C3E0855FF0A4FFAEF039
:102A430074081200398F738033856173802E856714
:102A53007380298568738024856973801F856A73F1
:102A6300801A856B73801585667380108565738006
:0C2A73000B856C738006900016E0F57374
:10395500022A31022A33022A38022A4C022A51024B
:103965002A56022A5B022A60022A65022A6A022A6C
:073975006F022A74022A7997
:102A7F009006D0E0FE9006D1E0D39E404B9006CF5B
:102A8F00E0B404189006D1E0C395735002D232908F
:102A9F0006D0E0D395734002C232802A9006D0E070
:102AAF00C3957350099006D1E0D3957350028002FD
:102ABF00D2329006D0E0D3957350099006D1E0C37F
:102ACF0095735002C232802A9006D0E0D39573409E
:102ADF00099006D1E0C3957340028002C23290067E
:102AEF00D0E0C3957340099006D1E0D395734002AF
:102AFF00D232229006D3E090397CF8282873804C8C
:102B0F0085537380479000C3E0855FF0A4FFAEF05C
:102B1F0074081200398F738033856173802E856737
:102B2F007380298568738024856973801F856A7314
:102B3F00801A856B73801585667380108565738029
:0C2B4F000B856C738006900016E0F57397
:10397C00022B0D022B0F022B14022B28022B2D02D3
:10398C002B32022B37022B3C022B41022B46022BF3
:07399C004B022B50022B55DA
:102B5B009006D4E0FE9006D5E0D39E404B9006D372
:102B6B00E0B404189006D5E0C395735002D23390AD
:102B7B0006D4E0D395734002C233802A9006D4E08A
:102B8B00C3957350099006D5E0D39573500280021C
:102B9B00D2339006D4E0D3957350099006D5E0C399
:102BAB0095735002C233802A9006D4E0D3957340BC
:102BBB00099006D5E0C3957340028002C23390069C
:102BCB00D4E0C3957340099006D5E0D395734002CA
:102BDB00D233229006D7E09039A3F8282873804C83
:102BEB0085537380479000C3E0855FF0A4FFAEF080
:102BFB0074081200398F738033856173802E85675B
:102C0B007380298568738024856973801F856A7337
:102C1B00801A856B7380158566738010856573804C
:0C2C2B000B856C738006900016E0F573BA
:1039A300022BE9022BEB022BF0022C04022C09025E
:1039B3002C0E022C13022C18022C1D022C22022C7A
:0739C30027022C2C022C311D
:102C37009006D8E0FE9006D9E0D39E404B9006D789
:102C4700E0B404189006D9E0C395735002D23490CB
:102C570006D8E0D395734002C234802A9006D8E0A4
:102C6700C3957350099006D9E0D39573500280023B
:102C7700D2349006D8E0D3957350099006D9E0C3B3
:102C870095735002C234802A9006D8E0D3957340DA
:102C9700099006D9E0C3957340028002C2349006BA
:102CA700D8E0C3957340099006D9E0D395734002E5
:102CB700D234229006DBE09039CAF8282873804C7A
:102CC70085537380479000C3E0855FF0A4FFAEF0A3
:102CD70074081200398F738033856173802E85677E
:102CE7007380298568738024856973801F856A735B
:102CF700801A856B73801585667380108565738070
:0C2D07000B856C738006900016E0F573DD
:1039CA00022CC5022CC7022CCC022CE0022CE502E8
:1039DA002CEA022CEF022CF4022CF9022CFE022D06
:0739EA0003022D08022D0D60
:102D13009006DCE0FE9006DDE0D39E404B9006DBA0
:102D2300E0B404189006DDE0C395735002D23590E9
:102D330006DCE0D395734002C235802A9006DCE0BE
:102D4300C3957350099006DDE0D39573500280025A
:102D5300D2359006DCE0D3957350099006DDE0C3CD
:102D630095735002C235802A9006DCE0D3957340F8
:102D7300099006DDE0C3957340028002C2359006D8
:102D8300DCE0C3957340099006DDE0D39573400200
:102D9300D23522AE2EAF2F74F5D39F74019E400817
:102DA300782E126492022EB0752F01752E00AE524A
:102DB300AF53E546BE000DD39F40099000A5E0D375
:102DC300954740028023754700E546C39553F57345
:102DD3009000A8E0D395454008E5452573F5458067
:102DE300069000A8E0F54580020547900081E0D3F6
:102DF3009561401CE55FC395604015AE52AF53E546
:102E030046BE00039F50099000A6E0D395484002B8
:102E1300806E9007C1E0A852B80004955350037523
:102E23004A009007C1E0A852B8000BD3955340065F
:102E3300E5539007C1F0E54A7041E553C39546F564
:102E430073E573D3940540037573059000A7E0C33E
:102E530095455007E573C3954540028009E545C391
:102E63009573F54580069000A7E0F5459000A7E02F
:102E7300D3954540069000A7E0F5457548008002CC
:102E83000548E54A7016900081E0C39561500DE551
:102E9300462405A852B8000695534002800F9000BF
:102EA30094E0F545754A0174789007C1F022AE2E7F
:102EB300AF2F74E9D39F74039E4008782E12649257
:102EC30002304F752F01752E00754532A236402A08
:102ED300754519900094E075F002A4FFAEF0E54744
:102EE300BE0006D39F4002D2360547754A03747865
:102EF3009007C1F075490002303EAE52AF53E5462C
:102F03006F4E700302303EE546BE000DD39F40096D
:102F13009000A5E0D395474002800F754700E54A2E
:102F2300C394035003754519800DE546C39553F5C6
:102F330073E5472573F547900081E0D39561400E13
:102F43009007C1E0A852B80007D395534002800C04
:102F53000549900094E0B54903754A00E54AB40376
:102F630006A20DB3B34002800A0549E549B43C0308
:102F7300754A02E54AB402299007C1E0A852B80095
:102F83000ED395534009E5539007C1F0754900905E
:102F93000081E0C39561500975490074789007C1B9
:102FA300F0E54A705A900081E0D39561401CE55FDB
:102FB300C395604015AE52AF53E546BE00039F5024
:102FC300099000A6E0D39548400280087548007533
:102FD300454B8028E553C39546F573E573D39405B4
:102FE3004003757305900081E0D395614008E5487F
:102FF3002573F5488006E5482406F548754900E53C
:103003004A7016900081E0C39561500DE546240592
:10301300A852B80006955340028003754A01E54A59
:10302300B401187545190549900094E0B549067532
:103033004A0275490074789007C1F0E54575F00AB6
:10304300A4FFAEF09007B2EEF0A3EFF022E56F908D
:1030530039F1F8282873900079E0700302327790F1
:1030630000AFE0B40102800302319290003CE0B56E
:103073005E02800302318F7E017F00E5BE12643E53
:10308300E5BD2FFF50010E8E5A8F5B741012643E04
:10309300900067E08E048F05FF12642E9007B6EC54
:1030A300F0A3EDF074FFBC00039D500B74FF900779
:1030B300B6F8E4F0E8A3F0E56B600FE56BC394FEAC
:1030C30050089000D5E06402600280649000C3E081
:1030D300B40B1F9007B6E0FEA3E0FF74E712643E53
:1030E300E56B8E048F05FF12642E9007B6ECF0A3F8
:1030F300EDF09000C3E0D3940B40089000ABE06484
:10310300046002802B9007B6E0FEA3E0FF9007B8AF
:10311300E0FCA3E0FDEFD39DEE9C400D12648A908A
:1031230007B6EEF0A3EFF080079007B6E4F0A3F044
:10313300900079E0B4021E9007B6E0FEA3E0FF9092
:1031430007C2E02FFF50010E74011200399007B639
:10315300EEF0A3EFF09007B6E0FEA3E0FF9007C206
:10316300E0BE0008D39F4004D2398002B2399007F1
:10317300B7E09007C2F09000ABE064016006A239AB
:10318300B3B3400280069007B7E0F55F023275D211
:10319300397E017F00E5BE12643EE5BD2FFF50017D
:1031A3000E8E5A8F5B741012643E900067E08E049B
:1031B3008F05FF12642E9007B6ECF0A3EDF0E56BDC
:1031C300600FE56BC394FE50089000D5E064026085
:1031D3000280649000C3E0B40B1F9007B6E0FEA327
:1031E300E0FF74E712643EE56B8E048F05FF126403
:1031F3002E9007B6ECF0A3EDF09000C3E0D3940B50
:1032030040089000ABE064046002802B9007B6E0B6
:10321300FEA3E0FF9007B8E0FCA3E0FDEFD39DEE33
:103223009C400D12648A9007B6EEF0A3EFF080077E
:103233009007B6E4F0A3F0900079E0B4021E900783
:10324300B6E0FEA3E0FF9007C2E02FFF50010E742B
:10325300011200399007B6EEF0A3EFF09007B7E044
:103263009007C2F09000ABE0640160069007B7E0FE
:10327300F55F8003755F00900075E07006756F0160
:1032830002305075BB18023845900075E070030298
:1032930033FD7E017F00E5BE12643EE5BD2FFF5086
:1032A300010E8E5A8F5B9000BBE0B4010F7E0F7F3F
:1032B300FFAC5AAD5B12648A8E5A8F5B9000E0E0DC
:1032C300B40245AE5AAF5B90001FE0FCA3E0FDEDF6
:1032D300D39FEC9E400A90001FE55AF0A3E55BF0F4
:1032E300AE5AAF5B900021E0FCA3E0FDEFD39DEE6F
:1032F3009C400A900021E55AF0A3E55BF0AE5AAF7B
:103303005B74041200398F619000E0E0704CAE5A98
:10331300AF5B90001FE0FCA3E0FDEFD39DEE9C406C
:103323000912648A8E5A8F5B8006755B00755A009A
:10333300AE5AAF5B741012643E900064E08E048F4B
:1033430005FF12642E8C5A8D5B74FFBC0009D39D5C
:103353004005855B6180037561FE9000ABE0B401BD
:103363000280030233FBA20DB3B3500E90007FE043
:10337300A852B80005D39553500280719000BCE069
:103383008561F0A4FFAEF074648E048F05FF1264B0
:103393002E8C5A8D5BE56B6016E56BC394FE500F64
:1033A3009000D5E0B402089000C3E0640B60028093
:1033B30017AE5AAF5B74E712643EE56B8E048F055C
:1033C300FF12642E8C5A8D5BAE5AAF5B9007B6E04A
:1033D300FCA3E0FDEDD39FEC9E4005855B5F800B76
:1033E300A239B340069007B7E0F55F800BA239B36B
:1033F30040069007B7E0F55F8003756100900078A1
:10340300E07006756F0202305075BB1902384590A3
:103413000078E070030234B2E55ED39551400302B5
:1034230034B090001DE0FEA3E0FFE56512648290D6
:10343300001DEEF0A3EFF07E017F00E5BE12643EB7
:10344300E5BD2FFF50010E8E5A8F5B9000E5E070B3
:1034530013740A12643E74518E048F05FF12642E96
:103463008D658019AE5AAF5B740A12643E8F048E69
:10347300057E017F95CDCCCD12632C8F65E565D399
:103483009464400375656490001DE0FEA3E0FFE5CE
:10349300652FFF50010E90001DEEF0A3EFF090009A
:1034A3007CE0048E048F05FF12642E8D6580037506
:1034B30065329000C8E07006756F0302305075BB2B
:1034C300130238459000C8E0604A7E017F00E5BEE4
:1034D30012643EE5BD2FFF50010E8E5A8F5B7404BC
:1034E3001200398F669000CAE08566F0A4FDACF047
:1034F3007464FF12642E8D669000C9E08566F0A4A3
:10350300FFAEF074FF8E048F05FF12642EED900062
:1035130063F08003756600900076E07006756F04B3
:1035230002305075BB17023845900076E0B40102B3
:1035330080030235C07E017F00E5BE12643EE5BD17
:103543002FFF50010E8E5A8F5B9007C3E0601990D6
:1035530007C3E014905D9E12008CE493FC74019306
:10356300FDEDC39FEC9E400280069007C3E014F07C
:103573009007C3E0C394B3501DAE5AAF5B9007C32B
:10358300E004905D9E12008CE493FC740193FDEFC4
:10359300C39DEE9C400280069007C3E004F09007B1
:1035A300C3E0FE90009CE08E0088F0A4FFAEF074B0
:1035B300648E048F05FF12642E8D67800375670088
:1035C300900077E07006756F0502305075BB1602E8
:1035D3003845900077E0B4010280030236697E012A
:1035E3007F00E5BE12643EE5BD2FFF50010E8E5AEB
:1035F3008F5B9007C4E060199007C4E014905F08E4
:1036030012008CE493FC740193FDEDC39FEC9E4088
:103613000280069007C4E014F09007C4E0C394B39B
:10362300501DAE5AAF5B9007C4E004905F081200D0
:103633008CE493FC740193FDEFC39DEE9C400280E8
:10364300069007C4E004F09007C4E0FE9000A2E0F7
:103653008E0088F0A4FFAEF074648E048F05FF1211
:10366300642E8D68800375680075BB1F0238457E24
:10367300017F00E5BE12643EE5BD2FFF50010E8EB3
:103683005A8F5B740912643E74E68E048F05FF1231
:10369300642E8D6A90007EE07006756F07023050CD
:1036A30075BB1502384590007EE070030237C47E77
:1036B300017F00E5BE12643EE5BD2FFF50010E8E73
:1036C3005A8F5B74041200398F6990007EE0B40155
:1036D300159000D2E08569F0A4FFAEF074071200E4
:1036E30039EF9007BBF090007EE0B402159000D252
:1036F300E08569F0A4FFAEF07407120039EF90077C
:10370300BAF090007EE0B4030280030237A7900072
:10371300BFE0701CE569C394195002D22BE569D34D
:1037230094644002C22B90009EE09007BEF0806339
:1037330090009EE070349000D2E08569F0A4FFAE63
:10374300F074FF8E048F05FF12642EED9007BEF018
:10375300AE52AF53741EBE0006D39F4002D22BE578
:1037630061D394E54002C22B8029E569C3940A50D2
:103773000DAE52AF53741EBE0004D39F500280029D
:10378300D22BE561D394E54002C22B90009EE090DA
:1037930007BEF09007BEE0C394055006740590077A
:1037A300BEF0C23A90007EE0B40414E569C39419F4
:1037B3005002D23AE569D394324002C23AC22B8016
:1037C300037569009000D5E07006756F08023050EC
:1037D30075BB14806D9000D5E060567E017F00E5D7
:1037E300BE12643EE5BD2FFF50010E8E5A8F5BEF74
:1037F300D39421EE940E4005756BFF8015AE5AAF3E
:103803005B741012643E74E38E048F05FF12642E02
:103813008D6BE56B75F00BA4FFAEF09000C3E08EEB
:10382300048F05FF12642E9007B8ECF0A3EDF0802F
:1038330003756B00900079E0600575BB1A80037512
:02384300BB18B0
:1039F10002305902328C0234120234C702352C02D1
:0B3A010035D50236720236A90237D814
:05384500056FD2EC222A
:096470002582F582500205832209
:0F008C0025E050020583258250020583F582226C
:10640D00EF2F500205832582F582E5833E2EF5831D
:01641D00225C
:10648200CFC39FFF50011E22C3EF9DFFEE9CFE2251
:086492000806B60002180622FC
:0D644C00A3E004F07006120049E004F02205
:0E003900048007C3CE13CECF13CFD5E0F6223E
:10632C00BC000FBE0008ED8FF084FFADF022E4FE40
:10633C00FF22BE000DEF60FE54F0606F20E70302F9
:10634C0063E2EAC0E0EBC0E078017A0075F001EEA0
:10635C0020E710EF25E0FFEE33FE0AC5F023C5F071
:10636C0030E7F0EA5407F9096A7A007B006001080B
:10637C00C3EC9E40167004ED9F4010ED9FFDEC9E0B
:10638C00FCE5F0CA4ACA03F5F08005E5F003F5F028
:10639C00C3EE13FEEF13FFD9D77908CACBCAD8D0F6
:1063AC00EAFEEBFFD0E0FBD0E0FA22EC8FF084FCAD
:1063BC00ED54F045F0C48FF084FEEDC454F045F07C
:1063CC00C48FF084FDEEC4FE54F02DFFEE540F3C50
:1063DC00FEADF07C0022790078008FF0EC7E082076
:1063EC00E70DC3CD33CD33C933C9C833C8DEF08410
:1063FC0049F9E5F08FF0BE00E6FD7C00E9FFE8FE10
:01640C00226D
:0E643E00F88FF0A4FFE5F0CE88F0A42EFE2229
:10000300EF8DF0A4F9A8F0EF8CF0A428F8EE8DF0B2
:06001300A428FEE9FF2213
:10641E00600D782B026428007830D8FED5E0F82283
:10642E00EEC0E07E0012632CEFFDEEFCD0E0FE220B
:0C645900EEC0E07E0012632CD0E0FE22BA
:03001B0002001EC2
:0300530002005652
:03009B00020071EF
:030000000264791E
:0964790075817575D00002422CFA
:0B646500E5822FF582E5833EF58322DF
:0A0049000582D5820215831582227C
:10001E00C0E0C0F0C083C082C0D075D0001241666F
:0B002E00D0D0D082D083D0F0D0E032E0
:10005600C0E0C0F0C083C082C0D075D00012416934
:10006600D0D0D082D083D0F0D0E032C0E0C0F0C093
:1000760083C082C0D075D0001241EED0D0D082D0DD
:0600860083D0F0D0E0324F
:00000001FF
